:020000040000FA
:20000000DCEF03F01200FFFF04EF04F01200FFFFFFFFFFFFFFFFFFFF0CEF04F01200FFFF24
:20002000FFFFFFFFFFFFFFFFFFFF0100D00700007E000000020000000001776B1E0E716E84
:200040000401400E096F200E0A6F040E0B6F880E086F0401200E0E6F040E0F6F400E0C6F8C
:200060001200550EA76EAA0EA76EA68212000401226B010E236F12000001756B5CD90AE2A8
:2000800067D90800F5CF76F000014ED976C0EFFF752BF4D7F86A1200F00E04012217840EF5
:2000A000A66E0001756B47D90AE24AD90F0E000175150F0801E1D5DF0001752BF4D7120049
:2000C000940EA66E0001756B36D911E27551006E016A060ED89000360136E804FBE1026ACB
:2000E00001BE026812D9BDDF0001752BEDD7F86A1200A66A0001756B1ED90BE2040122512A
:2001000000017525A96EA6800FD9A8CFEFFF752BF3D712000001756B0ED910E2040122510C
:2001200000017525A96E00D9EF50A86E040EA66E98DFA6B2FED70001752BEED71200C40ECB
:20014000A66E0001756BF7D805E2FAD88ADF0001752BF9D7F86A120097D8060E00017A5D79
:2001600003E36D50020B01E08ED00001770511E104010CBF0DD00401400E096F400E040156
:2001800008170401087D880E040108130001776B7AD0040108BF77D00001756B0401205169
:2001A000320A45E0CD0A34E0F80A2DE0020A26E0010A1FE0070A18E0010A11E0030A0AE0CC
:2001C000070A08E0060A01E04DD051DF0001040E756F49D051DF050E0001752744D05CDFA9
:2001E0000001010E756F3FD06BDF0001010E756F3AD07FDF050E0001752735D08BDF000136
:20020000010E756F30D09BDF0001010E756F2BD06D960001786B796B00017807000E795B55
:2002200000017851791101E0F7D7FF001CD0030E0401215D09E104012251E8B08C84E8A0AA
:200240008C940001010E756F040E0401215D09E104012251E8B08C86E8A08C960001010E2F
:20026000756F01D000D00001010E776F000175510AE075C00DF4400E04010C1704010C7D18
:20028000880E04010C13120000017E517F1104E1200E7E6F4E0E7F6F7E07000E7F5B6DA26C
:2002A00008D07E517F1130E18C708C50010B1CE128D000017A5102E18C8016D07A0502E11A
:2002C0008C901FD0020E7A5D02E18C900DD0030E7A5D02E18C8015D0050E7A5D07E10001C1
:2002E0007E517F1111E18C708C821200060E7A5D0BE100017E517F1107E18C708C50010B8E
:2003000002E08C9212008C821200040122510024F36E23510120F46E24510220F86EF4CFF7
:20032000F7FFF3CFF6FF12007551EA6A250FE96E040EEA221200040121510001755D1200CD
:20034000F3DFEFCF03F004D803C0F5FF0C00120075C000F0016A026A85EF01F06C5002E06A
:20036000000E01D0010E00090BE0040100513C0BE842E8420D0802E1C9EF01F0D2EF01F057
:200380006C5002E0000E01D0010E040901E019D812000001606B616B666B676B9DEC02F02A
:2003A00054EF02F0020E0001605D09E15CD8040100BD02D0C80E01D0880E006F12008DEF4E
:2003C00002F0040E00017A5D09E112C46EFF6E50000802E2050E01D0030E7A6F0001600526
:2003E00009E10AD8040104BD02D0C80E01D0880E046F12008DEF02F00001080E665D000E81
:20040000675903E266C069F002D0080E696F69C005F46951006E016A0050665F0150675B1B
:20042000180E646F040E656F69511CE000017BA307D062C0F6FF63C0F7FF0800F55005D0DF
:2004400062C0E9FF63C0EAFFEF5064C0E9FF65C0EAFFEF6E0001622B000E6323642B652397
:200460006907E2D7120001C46AF000016A516625666F000E6721676F180E626F040E636FBF
:200480006A5111E062C0E9FF63C0EAFFEF5064C0E9FF65C0EAFFEF6E642B000E6523622B32
:2004A00063236A07EDD712000001615105E13DD8840E006F04011DD0040110AF1CD000011D
:2004C00066510401165D000167510401175904E216C466F017C467F08FDF0001010E606F2A
:2004E00024D8800E006F0401180E066F040E076FC80E046F10D00001020E606F0401056B5D
:20050000C80E046F0401080E016F180E026F040E036FC80E006F6D9812000001606B05D8E7
:20052000880E006F0401046B12000401080E016F100E026F040E036F120004011051600BAF
:20054000E842E842E842E842E842000901E012001151080A39E0010A35E00F0A0AE0030A10
:2005600001E012000001010E616F0001040E7A6F12000001010E616F0401130507E10001B4
:200580004E0E626F070E636F120E13D0020E135D07E10001600E626F070E636F200E09D0AE
:2005A000030E135D0AE10001800E626F070E636F040E0001666F676B02D00001616B00012E
:2005C0007B831200F2EF02F00001010E616F00017C0E626F000E636F00017B930001010EFD
:2005E000666F12000001010E616F12C47CF00401125104E10001050E7A6F12000001060E81
:200600007A6F1CEF00F0080E6D6E6DBAFED7686A110E696E0001020E7A6F12006850040B6E
:2006200006E06950040B03E06D92699468946850010B04E06950010B01E027D86850100B11
:2006400009E06950100B06E0698468986D82A08A0300A19A6850200B09E06950200B06E01D
:2006600070A003D08DEC02F07090689A030E00017A5D01E209D06850080B06E06950080B08
:2006800003E0AEEC01F068961200686A7B0E696E6E6A160E706E68A602D06896FCD76D981A
:2006A0008DEC02F000017C6B0001030E7A6F12002A0EF66E000EF76E000EF86E000109004D
:2006C000F550706F0900F550716F03E1706701D03DD00900F5506B6F0900F5506C6F0900D5
:2006E000F5506D6F09000900F550E96E0900F550EA6E090009000900F5506E6F0900F550FA
:200700006F6F09000900F6CF72F0F7CF73F0F8CF74F06BC0F6FF6CC0F7FF6DC0F8FF000107
:200720006E5302E16F5307E00900F550EE6E6E07F8E26F07F9D772C0F6FF73C0F7FF74C0A9
:20074000F8FF00017007000E715BBFD712001201000200000008D8040B00000000000001A3
:2007600009022000010100803209040000020000000007050102400000070581024000006D
:2007800004030904C1CF80F00F0EC11282A204D080C0C1FF00EF04F0F00E8C12F00E951635
:2007A00094908B90140E6F6E03EC03F00EEC03F0ACEC00F0FBD7120013EE00F023EE00F0CE
:2007C000F86A059C58EC03F0C2EC03F0FDD712000000FFFFFFFFFFFFFFFFFFFFFFFFFFFF66
:2007E000FFFFFFFFFFFFFFFFFFFFFFFFFFFFFFFFFFFFFFFFFFFFFFFFFFFFFFFFFFFFFFFF19
:20080000FCEF0BF0FFFFFFFFFEEF0BF0E153D8A40BEF04F01200FF0E000000000000000051
:200820000000000000000000000000000000000000000000000000000000000000000000B8
:20084000000000000000000000000000000000000000000000000000000000000000000098
:200860000000000000000000000000000000FF0FD8A40CEF04F000000000000000000000FF
:200880000000000000000000000000000000E12F0BEF04F01200EB6BED6BEC6BECB712008E
:2008A000D890ED37E937EB37EB51EA6501D003D0EA51EB5FED81EC2BF1D7E75303E1030E3A
:2008C000E86F31D0E70503E19F0EE86F2CD0020EE76303D0250EE86F26D0030EE76303D015
:2008E0000D0EE86F20D0040EE76303D0990EE86F1AD0050EE76303D0490EE86F14D0060EA9
:20090000E76303D0C10EE86F0ED0070EE76303D01F0EE86F08D0080EE76303D0010EE86F8F
:2009200002D0190EE86FE851E96F12000001BA29BA6F050EBA6346D0BA6BB969B651E96FCB
:20094000640EEA6F4BEC04F0ED51BB6F640EBB03F350E76FF450E86FE751B65DE96F0A0E1A
:20096000EA6F4BEC04F0ED51BF6F640EBB03F350E76FF450E86FE751B65DEB6F0A0EBF03A4
:20098000F350E96FF450EA6FE951EB5DC26FBB51E76F5DEC04F0E951BB6FBF51E76F5DECBA
:2009A00004F0E951BF6FB40504E1FE0EBF15BF6F03D0010EBF11BF6FC251E76F5DEC04F0A9
:2009C000E951C26FC70511E1060EB86101D002D0C76B0BD0B70505E1B96BBB6BBF6BC26BCE
:2009E00004D0B969BB69BF69C269C05307E0C051E76F5DEC04F0E951B96F01D0B969BA538A
:200A000013E1FB0E9614966EFB0E8414E76F040EE711846E956ABE51836EFE0E9414946E83
:200A2000FE0E8214826E53D0BA0513E1FE0E9414946EFE0E8214E76F010EE711826E956AAA
:200A4000B951836EFB0E9414946EFB0E8214826E3ED0020EBA6313D0FB0E9414946EFB0E7F
:200A60008214E76F040EE711826E956ABB51836EEF0E9314936EEF0E8114816E28D0030E65
:200A8000BA6313D0EF0E9314936EEF0E8114E76F100EE711816E956ABF51836EEF0E921421
:200AA000926EEF0E8014806E12D0EF0E9214926EEF0E8014E76F100EE711806E956AC25135
:200AC000836EFB0E9614966EFB0E8414846EC529C56F250EC5631200C56BB729B76F010E07
:200AE000B715B76FB829B86F040EBC631200572AD8B4582A5E5000085B6E010E5C6ED8A05A
:200B00005C065850800AE76F5C50800AE75D04E157505B6401D01200D8A01200576A586A36
:200B2000C029C06F050EC0631200010EC06F1200E051E46FE135E133E431E06FE26BE36B58
:200B4000E351800AE46FE151800AE45D02E1E051E25DD8B01200000000000000000000009A
:200B600000000000000000000000E24BE32BE8D7650EAC6E0B0EAF6EAB6AAB8E7F0E941435
:200B8000946E12009EA8FED7E051AD6E12000001C0051EE1010E596E5A6ADF6B280EDF61A9
:200BA0001200000EEA6E050EE96E5950E926EF50E26F0101010EEA6E000EE96E5950E92685
:200BC0000001E251EF6E592AD8B45A2ADF2BE6D7020EC0631ED0010E596E5A6ADE6B280EF0
:200BE000DE611200000EEA6E2E0EE96E5950E926EF50E26F0101010EEA6E000EE96E5950EC
:200C0000E9260001E251EF6E592AD8B45A2ADE2BE6D7030EC0631ED0010E596E5A6ADD6BD7
:200C2000280EDD611200000EEA6E600EE96E5950E926EF50E26F0101010EEA6E000EE96EED
:200C40005950E9260001E251EF6E592AD8B45A2ADD2BE6D7040EC0631200010E596E5A6A12
:200C6000DC6B280EDC611200000EEA6E890EE96E5950E926EF50E26F0101010EEA6E000E95
:200C8000E96E5950E9260001E251EF6E592AD8B45A2ADC2BE6D7E2290BE0E25305E0E22942
:200CA000E36FE205E46F07D0E229E36FE46B03D0E369E205E46FE151E36103D0010EE56F20
:200CC00007D0E451E16103D0010EE56F01D0E56BE551E66F1200010E596E5A6A0001DB6BF1
:200CE000280EDB6112000101010EEA6E000EE96E5950E926000EEF6E592AD8B45A2A0001EB
:200D0000DB2BEED7AB9E7F0E9414946E828EBF0E9414946EBF0E8214826E580E0001E06FF8
:200D2000E16B98EC05F0BF0E9414946EBF0E8214E06F400EE011826E080EE06FE16B98EC61
:200D400005F0829EAB8E1200030EC06E080EC16E96500001E16F020E9610966E190EC26E67
:200D6000E26B280EE26102D0E22BFBD7020EC210C26EC2B2FED7E151966E0F0EC16EC26AF3
:200D80001200C4500001E16F1200030EC06E090EC16E96500001E16F010E9610966E150E32
:200DA000C26EE26B280EE26102D0E22BFBD7020EC210C26EC2B2FED7E151966E0F0EC16EAF
:200DC000C26A1200C4500001E16F1200030EC06E0A0EC16E92500001E16F200E9210926ED5
:200DE000110EC26EE26B280EE26102D0E22BFBD7020EC210C26EC2B2FED7E151926E0F0E83
:200E0000C16EC26A1200C4500001E16F1200030EC06E0B0EC16E92500001E16F080E92107C
:200E2000926E0D0EC26EE26B280EE26102D0E22BFBD7020EC210C26EC2B2FED7E151926E63
:200E40000F0EC16EC26A1200C4500001E16F1200030EC06E0C0EC16E92500001E16F040EC4
:200E60009210926E090EC26EE26B280EE26102D0E22BFBD7020EC210C26EC2B2FED7E15185
:200E8000926E0F0EC16EC26A1200C4500001E16F1200030EC06E0D0EC16E92500001E16F95
:200EA000020E9210926E050EC26EE26B280EE26102D0E22BFBD7020EC210C26EC2B2FED76B
:200EC000E151926E0F0EC16EC26A1200C4500001E16F1200030EC06E0E0EC16E9250000172
:200EE000E16F010E9210926E010EC26EE26B280EE26102D0E22BFBD7020EC210C26EC2B2B5
:200F0000FED7E151926E0F0EC16EC26A1200C4500001E16F12000001C4691F0E9314936EC6
:200F20001F0E8114E16FC00EE111816E010EE16F06EC04F00F0E9310936E0F0E8114E06FE9
:200F40000E0EE06303D0010EC46F11D00D0EE06303D0040EC46F0BD00B0EE06303D0070EA7
:200F6000C46F05D0070EE06302D00A0EC46F1F0E9314936E1F0E8114E16FA00EE111816E7E
:200F8000010EE16F06EC04F00F0E9310936E0F0E8114E06F0E0EE06303D0020EC46F11D0F4
:200FA0000D0EE06303D0050EC46F0BD00B0EE06303D0080EC46F05D0070EE06302D00B0E4F
:200FC000C46F1F0E9314936E1F0E8114E16F600EE111816E010EE16F06EC04F00F0E9310A3
:200FE000936E0F0E8114E06F0E0EE06303D0030EC46F11D00D0EE06303D0060EC46F0BD045
:201000000B0EE06303D0090EC46F05D0070EE06302D00C0EC46F1F0E9314936E1F0E811474
:20102000E16FE00EE111816EC151C463C16303D0C451BD6F01D0BD69C451C16F12000001D1
:20104000BA6BBF0EBE6FB66BBC6BC76BC86BC06BC36BD59AD588F00ED514E06F060EE01164
:20106000D56EF28EF28AB8EC05F0596A5A6AC10E59605A665A6601D002D05AAE0DD001017F
:20108000010EEA6E000EE96E5950E926000EEF6E592AD8B45A2AEBD7596A5A6A0001D86B41
:2010A000290ED8611200000EEA6E050EE96E5950E926000EEF6E000EEA6E2E0EE96E595019
:2010C000E926000EEF6E000EEA6E600EE96E5950E926000EEF6E000EEA6E890EE96E59504B
:2010E000E926000EEF6E592AD8B45A2AD82BD8D70001BC5316E10B0EBD6303D0010EBC6FE4
:2011000036D00C0EBD6307D0040EBC6F576A586A010EC06F2CD0090EBD6329D0030EBC6F52
:2011200026D0BC050CE10B0EBD6303D0030EBC6F1ED00A0EBD631BD0020EBC6F18D0030E7E
:20114000BC6306D0090EBD6312D0BC6BC06B0FD0040EBC630CD00C0EBD6303D0BC6BC06BE4
:2011600006D0090EBD6303D0030EBC6FC06BE16BBC05D8B4E12BE06B020EBC6301D0E02B2D
:20118000E051E1110AE0B70504E1FB0EBE15BE6F1BD0040EBE11BE6F17D0030EBC6307D0B1
:2011A000FD0EBE15BE6F050EBE11BE6F0DD0040EBC6307D0FE0EBE15BE6F060EBE11BE6F14
:2011C00003D0070EBE11BE6FBD050CE1E369BE1DE26F080EE215E46FE56BF70EBE15E41187
:2011E000BE6F37D0020EBD630CD0E369BE1DE26F100EE215E46FE56BEF0EBE15E411BE6F8D
:2012000028D0030EBD630CD0E369BE1DE26F200EE215E46FE56BDF0EBE15E411BE6F19D0BE
:20122000080EBD6316D0E369BE1DE26F400EE215E46FE56BBF0EBE15E411BE6FE369BE1D49
:20124000E26F800EE215E46FE56B7F0EBE15E411BE6F040EBC6303D0C7EC05F06DD1030E98
:20126000BC6303D06BEC06F067D1380EBE15E26F380EE263B6D0BC53D8A45ED1040EBD6390
:2012800029D0C80505E16BEC06F0C86BC06B54D1010E596E5A6AD36B280ED36117D0000E9B
:2012A000EA6E050EE96E5950E926EF50E36F0101010EEA6E000EE96E5950E9260001E35168
:2012C000EF6E592AD8B45A2AD32BE6D7010EC86FC06F32D1050EBD632AD0020EC86305D0AE
:2012E0006BEC06F0C86BC06B27D1010E596E5A6AD26B280ED26117D0000EEA6E2E0EE96E2B
:201300005950E926EF50E36F0101010EEA6E000EE96E5950E9260001E351EF6E592AD8B45D
:201320005A2AD22BE6D7020EC86FC06F05D1060EBD632AD0030EC86305D06BEC06F0C86B64
:20134000C06BFAD0010E596E5A6AD16B280ED16117D0000EEA6E600EE96E5950E926EF5051
:20136000E36F0101010EEA6E000EE96E5950E9260001E351EF6E592AD8B45A2AD12BE6D7B7
:20138000030EC86FC06FD8D0070EBD63D5D0040EC86305D06BEC06F0C86BC06BCDD0010EEB
:2013A000596E5A6AD06B280ED06117D0000EEA6E890EE96E5950E926EF50E36F0101010E6B
:2013C000EA6E000EE96E5950E9260001E351EF6E592AD8B45A2AD02BE6D7040EC86FC06F43
:2013E000ABD0020E9410946E020E8214E36FB56B020EE36301D0B52BB5530BE1010EC311C6
:20140000C36FC30506E1B45303E1010EB46F01D0B46BC351E36FD890E335C36F030EC315DD
:20142000C36FBEB731D0BEBD20D0B4050EE1C9510101016F0001CA510101026F0001CD51B7
:201440000101036F5D50046F1FD0C9510101016F0001CA510101026F0001CC510101036F5C
:201460000001CF510101046F0FD0C9510101056F0001CA510101066F0001CC510101076F3E
:201480000001CF510101086F0001BEB931D0BEBD20D0B4050EE1CD510101116F5D50126F58
:2014A0000001CC510101136F0001CF510101146F1FD0C9510101116F0001CA510101126FBA
:2014C0000001CC510101136F0001CF510101146F0FD0C9510101156F0001CA510101166FA2
:2014E0000001CC510101176F0001CF510101186F0001BEBB21D0BEBD10D0C9510101216F2A
:201500000001CA510101226F0001CC510101236F0001CF510101246F0FD0C9510101256F25
:201520000001CA510101266F0001CC510101276F0001CF510101286F020E0001BC63120046
:20154000040EBD6325D0010E596E5A6AD76B280ED76117D00101010EEA6E000EE96E5950BC
:20156000E926EF500001E26F000EEA6E050EE96E5950E926E251EF6E592AD8B45A2AD72B1E
:20158000E6D7010EBC6FC76FB86B010EC06F1200050EBD6325D0010E596E5A6AD66B280E72
:2015A000D66117D00101010EEA6E000EE96E5950E926EF500001E26F000EEA6E2E0EE96EFD
:2015C0005950E926E251EF6E592AD8B45A2AD62BE6D7010EBC6FC76FB86B020EC06F12008E
:2015E000060EBD6325D0010E596E5A6AD56B280ED56117D00101010EEA6E000EE96E59501E
:20160000E926EF500001E26F000EEA6E600EE96E5950E926E251EF6E592AD8B45A2AD52B24
:20162000E6D7010EBC6FC76FB86B030EC06F1200070EBD631200010E596E5A6AD46B280EB2
:20164000D46117D00101010EEA6E000EE96E5950E926EF500001E26F000EEA6E890EE96E03
:201660005950E926E251EF6E592AD8B45A2AD42BE6D7010EBC6FC76FB86B040EC06F1200ED
:201680006AEC07F087EC07F0E151C96F49EC07F066EC07F0E151CA6F28EC07F045EC07F016
:2016A000E151CC6F07EC07F024EC07F0E151CF6FE6EC06F003EC07F0E1515E6EC5EC06F009
:2016C000E2EC06F0E151CD6FA4EC06F0C1EC06F0E1515D6EC951E16FCB51E26F4BEC06F0AE
:2016E000E651C66FC60503E1010EB36F26D0CA51E16FCE51E26F4BEC06F0E651C66FC60569
:2017000003E1020EB36F19D0CC51E16F5F50E26F4BEC06F0E651C66FC60503E1030EB36FE2
:201720000CD0CF51E16FB251E26F4BEC06F0E651C66FC60502E1040EB36F380EBE15E06F26
:20174000380EE06308D0040EBC6303D05B50B66F18D0B66B16D0B30503E1C951B66F11D0A9
:20176000020EB36303D0CA51B66F0BD0030EB36303D0CC51B66F05D0040EB36302D0CF512A
:20178000B66FC951CB6FCA51CE6FCC515F6ECF51B26F120082EC06F0596A5A6AD96B0C0EF2
:2017A000D9611200DA6B100EDA6111D00101010EEA6E000EE96E5950E926EF500001E06F49
:2017C000C2EC05F0592AD8B45A2ADA2BECD7020EE16F06EC04F0D92BE2D70F0EC16E080EA6
:2017E0006F6E1FEC08F040EC0BF08BEC07F078EC08F0CAEC0BF0F7D7EDEF0BF0EACF01F018
:20180000E9CF02F0F4CF03F0F3CF04F0F2A403D096EC04F0F29404C0F3FF03C0F4FF02C01F
:20182000E9FF01C0EAFF1100FFFFFFFFFFFFFFFFFFFFFFFFFFFFFFFFFFFFFFFFFFFFFFFF1D
:20184000FFFFFFFFFFFFFFFFFFFFFFFFFFFFFFFFFFFFFFFFFFFFFFFFFFFFFFFFFFFFFFFFA8
:20186000FFFFFFFFFFFFFFFFFFFFFFFFFFFFFFFFFFFFFFFFFFFFFFFFFFFFFFFFFFFFFFFF88
:20188000FFFFFFFFFFFFFFFFFFFFFFFFFFFFFFFFFFFFFFFFFFFFFFFFFFFFFFFFFFFFFFFF68
:2018A000FFFFFFFFFFFFFFFFFFFFFFFFFFFFFFFFFFFFFFFFFFFFFFFFFFFFFFFFFFFFFFFF48
:020000040020DA
:020000040030CA
:0E000000E43EFFFEFFF99BFFFFFFFFBFFFFF87
:00000001FF
